:1000000060220020C91B0000C51B0000C51B0000AA
:1000100000000000000000000000000000000000E0
:10002000000000000000000000000000C51B0000F0
:100030000000000000000000C51B0000C51B000000
:10004000C51B0000C51B0000C51B0000C51B000030
:10005000C51B0000C51B0000C51B0000C51B000020
:10006000C51B0000F9140000091500001915000057
:10007000291500003915000049150000C51B0000B6
:10008000C51B0000C51B0000C51B0000C51B0000F0
:10009000C51B0000C51B0000C51B0000C51B0000E0
:1000A000C51B0000C51B0000C51B0000C51B0000D0
:1000B0000000000010B5064C2378002B07D1054B3B
:1000C000002B02D0044800E000BF0123237010BDC4
:1000D0006800002000000000404A0000084B10B5F6
:1000E000002B03D00749084800E000BF0748036819
:1000F000002B00D110BD064B002BFBD09847F9E731
:10010000000000006C000020404A0000404A00004F
:100110000000000001680722CB691A42FCD1704739
:10012000F0B5D6464F464646C0B58AB006000F0029
:10013000140031600800A04B9847A04A116A851C42
:100140000123AB400B43136209A9237B0B701430CE
:10015000C5B228009A4B984728009A4B9847207BB5
:100160000021994B98473B681C209B0705D50AB096
:100170001CBC90469946A246F0BD3B681738DB0789
:10018000F5D430688C4B9946984705008F49904BC1
:100190009847AD008F4BEE500023337673760025E1
:1001A0007383B3832522B554336214333B603368C1
:1001B00098461800C8478146802308AA13705570D6
:1001C00001239370D570E069276A002800D1AFE061
:1001D00008AB1870022308AA5370000CC0B21100BB
:1001E0007D4B9847002F00D1A7E008AB1F7002237A
:1001F00008AA53703F0CF8B21100774B9847A38AB6
:10020000F380E38A3381237E8022002B04D1734B59
:100210009B789B07DB0FDA01A16823690B4313432B
:100220002422A25C002A02D08022D2051343A26AB3
:1002300013432C22A25C002A03D180229204914213
:1002400002D18022120513432D22A25C002A02D083
:100250008022120413432E22A25C002A02D08022A4
:10026000D20313434246126813434246136080236D
:100270005B00536048461430C0B2594B9847079012
:10028000FA239B0022685A43914663689A46554D6B
:10029000A847009001914B465800A847029003914F
:1002A000208EA847049005914F4F504A504B00981C
:1002B0000199B84702000B0004980599B8474D4EC4
:1002C00000224D4BB047049005914846A8470200D4
:1002D0000B0004980599B84702000B00474D0098A1
:1002E0000199A847029A039BB0470022444BA847B4
:1002F000029A039B434DA847434B98470500802330
:100300009B04A2689A421ED003004020FF2D00D912
:100310002DE700240020FF251D402406254300046E
:10032000FF231B04184005434346DD6000201EE701
:1003300000214046354B98474AE701214046334B60
:100340009847070051E7FA26B60053465E430098E7
:10035000019902000B00274CA0470090019130004A
:10036000204B984700222A4BB84702000B00009808
:100370000199244CA0470022214B204CA047224B3E
:100380009847041E0CD031000798224B984702383A
:10039000001B2B00FF2D0CD8FF28BCD94020E6E61F
:1003A0007100481E079B9C4660441A4B98470138D1
:1003B000EFE74020DBE6C046511400000004004097
:1003C0006D1A0000E11900008D120000A106000066
:1003D0008D14000044020020651B00000020004135
:1003E000891A0000CD360000392B000095D626E88A
:1003F0000B2E113EB11E00000000244039300000D9
:100400000000F03FD124000065360000D912000042
:1004100000000840451D000003681A7E920707D5BA
:1004200002221A765B8B9B074120DB17184070472E
:100430005A8B520706D55968C02292020A435A6065
:100440001820F4E70020F2E730B502680023012409
:100450000225117E21420BD1117E294206D10133A2
:100460009BB201899942F4D8122002E0002000E0FA
:10047000002030BD10B5046862688023DB0213439E
:1004800063606162024B98470123237610BDC0462A
:1004900049040000F0B5DE4657464E464546E0B5F5
:1004A00083B006000F0005684C88324B98477B7A72
:1004B000002B1DD16B68304A13406B603B7A002BD8
:1004C0001BD03B885B007A7A92031343802212028E
:1004D00013436B623000294B98470190002813D0DA
:1004E000019803B03CBC90469946A246AB46F0BD8D
:1004F000B97A3000224B9847DCE73B885B007A7A78
:10050000920313436B62E5E730001E4B9847031ECE
:100510000190E5D1A046002420339946154B9B4617
:10052000164B9A46444515D06B8B4A4613421DD054
:100530003000D8477B681A5D2823EA543000D04742
:10054000002806D16B8B01345B07EBD51E2301938A
:1005500000E00190B37A002BC2D03000054B9847E1
:100560006A68C0239B0213436B60B9E74123019380
:10057000B6E7C04615010000FFFFFBFF490400007D
:10058000750400001904000010B5838B9BB205228E
:10059000002B01D0100010BD01338372C372024BD7
:1005A00098470200F6E7C0469504000010B5838B1B
:1005B0009BB20522002B01D0100010BD83720133C5
:1005C000C372024B98470200F6E7C046950400004C
:1005D00001680722CB691A42FCD1704770B504004C
:1005E00006683268458B838BED1AADB2838B013B75
:1005F0009BB2838313011DD5C37A002B03D0838B59
:100600009BB2012B10D0A38B9BB2002B02D1A37AFB
:10061000002B1CD12000124B9847236A5D19282318
:10062000F35CDBB22B7070BD72688023DB02134376
:100630007360E8E7C37A002BE5D0838B9BB2002B75
:10064000E1D172688023DB0213437360DBE7200093
:10065000034B98477268C0239B0213437360D9E72A
:10066000D105000070B5040005686B8B5B0703D5EE
:100670001E222523C25470BD468B838BF61AB6B258
:10068000838B013B9BB28383044B9847236A9E195B
:100690003378DBB22822AB54EDE7C046D105000029
:1006A00070B58000754BC45825682B681B01DA0FA4
:1006B000637E267E1E40638B9BB2002B03D1A38BEF
:1006C0009BB2002B23D1638B9BB2002B08D0A38B52
:1006D0009BB2002B04D12533E35C052B00D16DE0E8
:1006E000638B9BB2002B24D0A38B9BB2002B20D01A
:1006F0006B8B9B0600D581E0002A04D0A38B9BB2B4
:10070000012B00D17AE041222523E25411E02B7E17
:10071000DB0707D501232B766B8B9B072ED5412258
:100720002523E254A38B9BB263832523E35C052B33
:1007300038D0638B9BB2002B07D0A38B9BB2002BCE
:1007400003D12533E35C052B64D02523E35C052B23
:1007500013D02523E35C002B0FD003232B7500233C
:100760006383A3832533E35C412B03D0A37A002B5F
:1007700000D075E0730700D57BE070BD6B8B5B0725
:10078000D0D518222523E2540023A383A37A002B7B
:10079000C8D020003A4B98476A68C0239B02134395
:1007A0006B60BFE71F33E35C002B03D02000354BA9
:1007B0009847BEE72000344B9847BAE71F33E35C05
:1007C000002B00D08CE703332B7500236383253384
:1007D0000022E254A37A002B07D101232B76F307E2
:1007E000A7D5E36820009847A3E72000244B98474B
:1007F0006A68C0239B0213436B60F0E72423E35C29
:10080000002B03D12000204B984792E720001D4B7E
:1008100098478EE71F33E35C012B96D12B7E9B0715
:1008200001D502232B7603232B7500236383253305
:100830000022E254B30703D52423E35C012B0BD041
:10084000F30700D481E72423E35C002B00D07CE78E
:10085000E3682000984778E723692000984774E709
:100860002000074B98476A68E023DB0213436B6064
:1008700080E76369200098477FE7C0464402002074
:10088000D1050000DD05000065060000F0B5C64694
:1008900000B50C00904600280FD1002A11DD8F18FA
:1008A000094E0A4D306821002B6898470134BC423C
:1008B000F8D1404604BC9046F0BD01235B42984607
:1008C000F7E78046F5E7C046D8000020D0000020BA
:1008D000F0B5C64600B50E0015000138022810D844
:1008E000002A11D000240C4B98460C4F4346186840
:1008F000315D3B689847002808DB0134A542F5D1FB
:1009000006E00124644203E0140001E00124644293
:10091000200004BC9046F0BDD8000020D400002088
:1009200070B51B4B00245D682C705C6821700178E9
:10093000198001215980002A14D11D00154C164E32
:1009400029002000B047002820D0144A1368591C01
:100950001160134A9342F3DD0022104B1A6001200C
:10096000404213E00A4D0B4C0E4E29002000B047C8
:1009700000280BD0094A1368591C1160084A934299
:10098000F3DD0022054B1A600120404270BDC046D5
:1009900004020020DC010020AD05000084000020DE
:1009A000CF0700008905000030B58FB001AB0022F1
:1009B00003921A731A768021890305910121494215
:1009C000D982998225315A540B9208315A540131F7
:1009D0005A5401315A54A93119861B4908911B49AF
:1009E0000991C821490001910292194B1949596096
:1009F000012159801A72184D184C01AA1849280073
:100A0000A0470028F9D1144B1C680722E3691A4259
:100A1000FCD123680222134323600F4D2868114B39
:100A200098471F2318401E3B83400F4A1360E888F5
:100A300000231021628B0A4204D101338342F9D38F
:100A4000102363830FB030BD0300080003000900CA
:100A500004020020DC000020DC0100202101000055
:100A600000100042C914000000E100E070B582B03F
:100A700005000E0000226B46DA80064C6B46991D7D
:100A80002800A0470028F9D16B4606331B88337035
:100A900002B070BD170F000070B505008CB2034E98
:100AA00021002800B0470028FAD170BDF10E0000E7
:100AB000F0B591B08023DB05009300230193FF2262
:100AC00069460A8100228B72CB7201242421684678
:100AD00044540131445401314354013143540A9385
:100AE000053143540131435405930382C3760276A2
:100AF000027742761323837642771E4B0C931E4B6C
:100B00000D9301235B420E930F9380235B030393AA
:100B1000E1235B020893194D194B1D60194A1A4BCA
:100B20001A601A4A1A4B1A606A461A4928001A4B68
:100B300098471A4F3B6898680021194EB0473B68A8
:100B400058680021B0472E683000164B98471F2385
:100B500018408440144B1C602A68D369002BFCD1D8
:100B600033680222134333601048114B984711B089
:100B7000F0BDC0460200160002001700100200205F
:100B8000D8000020990A0000D40000206D0A00005F
:100B9000D000002000140042B50B0000040000202B
:100BA000D9380000C914000000E100E088480000C6
:100BB000C5380000F0B5DE4657464E464546E0B51E
:100BC00091B005000C00160029600800BA4B984748
:100BD000020023680520DB0706D511B03CBC904617
:100BE0009946A246AB46F0BD236817309B07F4D464
:100BF000B249086A971C0123BB4003430B620FA94B
:100C00002D27F35D0B701432D3B202931800AC4B56
:100C100098470298AB4B9847F05D0021AA4B984744
:100C2000F37A6B712423F35CAB712523F35CEB71D6
:100C3000F37E2B72337F6B722B68984618009E4BA5
:100C40009847143000220E2306A98C4663441A806C
:100C5000328A02928023DB019A4200D19AE00FD9B6
:100C6000C023DB01029A9A4200D18EE080231B024E
:100C70009A4200D01BE1032306930023079308E068
:100C800080239B019A4200D011E1102306930F3B71
:100C9000079333680593F3689B4673690393337E28
:100CA00004932623F35C9A4673689946002B00D17F
:100CB0009CE080235B05994500D180E0737E002B8A
:100CC00002D0B37E424693730E2306AA9446634431
:100CD0001B8842469381059B5A461343039A13434C
:100CE0004A461343029F1F43049B1B021F43534664
:100CF0005B071F432723F35C002B01D104331F4301
:100D0000737E9B02327F52021343727F120213439F
:100D10002422B25C520413432522B25C1204134312
:100D2000B17AF27A114319433389FF2B00D181E064
:100D300080225204174319432C23F35C002B03D168
:100D4000624B9B789B0701D580231F432A68D36998
:100D5000002BFCD1434659602A68D369002BFCD193
:100D600043461F600EAB80221A7000225A70DA7060
:100D70009A70336B0A93736B0B93B36B0C93F36B97
:100D800002930D9300270AAE63E008230693073B06
:100D900007937EE733680593F3689B467369039373
:100DA000337E04932623F35C9A4673689946002B9E
:100DB00018D080235B05994501D0002025E027232A
:100DC000F35C002B00D079E7336A1F00C0B2404BC0
:100DD000984701000E2206AB9C46624438003D4B0A
:100DE000984712E008230693002307932723F35C18
:100DF000002B0ED0069B0093079B0E2206A98C4663
:100E00006244B16A306A344FB847002800D0E4E643
:100E100054E7336A1F00C0B22D4B98470100069B70
:100E20000093079B0E2206A88446624438002A4F8E
:100E3000B847EAE7F37E002B00D17DE78023DB048F
:100E40001F4379E72000254B984707E00137042F1F
:100E50000DD0F9B2BB0098590028F3D0431CF5D04F
:100E60000EA90870000CC0B21D4B9847EEE7002396
:100E7000EB602B616B61AB61EB612B62AB626B6210
:100E80000022EB85AB853033EA540133EA54013359
:100E9000EA540133EA542868074B98470400114983
:100EA000114B9847A400114BE550002095E6102304
:100EB000069300230793ECE6511400000004004061
:100EC0006D1A0000E11900008D12000000200041A1
:100ED000891A0000CF110000F9110000D91200009A
:100EE000651B0000810F00008D14000044020020EB
:100EF000C2791C23002A01D118007047C28D92B21A
:100F0000173B002AF8D1026811850221137E0B429B
:100F1000FCD00023F0E782791C23002A01D11800BD
:100F20007047828D92B2173B002AF8D10268107E7A
:100F30004007F4D5538BDBB298061DD0980703D534
:100F4000022353831833EAE7580703D50423538356
:100F50001A33E4E7D80703D5012353831233DEE7BE
:100F6000D80603D5102353833233D8E79B0603D525
:100F7000202353832133D2E7138D0B800023CEE748
:100F8000F8B58000624BC5582C68E369002BFCD192
:100F9000237EA67D1E403023EB5C3122AF5C1F40D8
:100FA000F30722D5EB8D9BB2002B1CD0AA6A1378D5
:100FB000DBB2511CA962697901290ED09BB2DB0515
:100FC000DB0D2385EB8D013B9BB2EB85002B0CD118
:100FD000013323750133A37507E0517809020B43F0
:100FE0000232AA62EBE701232375B30706D5022379
:100FF000237500223133EA54FB071AD4730765D5F1
:10100000AB8D9BB2002B5FD0638BDBB21A0714D47D
:101010003F221340002B34D09A0711D51A223223D5
:10102000EA54303B63837B0750D528006B699847AF
:101030004CE02800EB689847E0E737221340E9E7E7
:101040005A0705D51E223223EA542E3B6383EAE772
:10105000DA0705D513223223EA54313B6383E2E7F2
:10106000DA0605D542223223EA54223B6383DAE7CB
:1010700020221A42D7D021323223EA54123B638312
:10108000D1E7238DDB05DB0DDAB2696A0A706A6A83
:10109000511C69626979012910D0AB8D013B9BB26B
:1010A000AB85002B12D10433237500222E33EA5472
:1010B000BB070BD528002B69984707E01B0A537024
:1010C0006B6A01336B62E8E704232375F30604D5EA
:1010D000102323752376FB060ED4B30604D52023F4
:1010E000237523763B070BD4330704D508232375D8
:1010F0002376BB0608D4F8BD2800EB699847ECE7D7
:101100002800AB699847EFE72B6A28009847F2E779
:1011100044020020F0B5DE4657464E464546E0B54F
:1011200087B08046049116001F0000220023002192
:101130008B463F2401202100009601975C460394D2
:101140004446059413E02024641A0500E540A846AF
:1011500014E0009C019D121BAB415C464D462C43A4
:10116000A346039C45462C430394013925D32024F0
:1011700064420C19E7D40500A540A84604008C4041
:10118000A14692185B4114001D00059E4F463E404B
:10119000B446049E47463E40B246664657463E43E6
:1011A00003D00600264332002B00009C019D9D4287
:1011B000DBD8CED19442D8D8CBE7039B5846190050
:1011C00007B03CBC90469946A246AB46F0BD10B570
:1011D000490840230024814202D2180010BD1C009F
:1011E000091A631C9BB28842F9D94023FF2CF4D81A
:1011F00014800023F1E70000F0B583B00F00160063
:1012000008AA117804004C434022BC4202D91000C5
:1012100003B0F0BD002B14D1020008000021194CCE
:10122000A04701003A0000230020174CA0470022ED
:101230000123121A8B41120C1B041A433280002224
:10124000E5E70022012BF9D10A00002300210D4C13
:10125000A04702000B0000920193380000210A4CC5
:10126000A047050080239B0140229842CFD8790FE8
:10127000F800009A019BA047EA00821AD2B25203FA
:101280002A43DBE75D1E00001511000010B582B097
:1012900004000E4B1B78002B07D0002905D10B4B07
:1012A0005B78834210D01D200CE001A90C70132044
:1012B000074B98471320074B9847044B5C7001225B
:1012C0001A70002002B010BD0020FBE7880000204B
:1012D0006D1A0000E1190000404B984231D00AD944
:1012E0003F4B98424DD03F4B98425AD03E4B98428C
:1012F00037D0002070473D4B98420CD03C4B984271
:10130000F7D1012917D000295DD0022915D0032972
:1013100015D00020EEE7012907D0002951D002297D
:1013200005D0032905D00020E4E73248E2E732483F
:10133000E0E73248DEE73248DCE73248DAE73248B5
:10134000D8E7012907D000293FD0022905D0032979
:1013500005D00020CEE72D48CCE72D48CAE72D4820
:10136000C8E7012907D0002931D0022905D0032977
:1013700005D00020BEE72848BCE72848BAE728483F
:10138000B8E7012907D0002923D0022905D0032975
:1013900005D00020AEE72348ACE72348AAE723485E
:1013A000A8E7012907D0002915D0022905D0032973
:1013B00005D000209EE71E489CE71E489AE71E487D
:1013C00098E71E4896E7032094E71D4892E71D48DA
:1013D00090E71D488EE71D488CE7C046001000428C
:1013E00000180042001C00420014004200080042A5
:1013F000000C004203000500030006000300070084
:101400000300010003001E0003001F000300090089
:1014100003000A0003000B00030011000300120088
:101420000300130003000D0003000E0003000F0073
:101430000300170003001800030019000300040054
:10144000030008000300100003000C000300160056
:1014500030B587B00B4B6A4632CB32C232CB32C288
:10146000009B83420BD001239A0069465258824266
:1014700006D00133062BF7D1002007B030BD002382
:10148000D8B2FAE79448000070470000F0B50A4B64
:101490001B78002B0CD1094F094E0A4D0024DE5158
:1014A0005A1914600433182BF9D10122024B1A7017
:1014B0008000024BC150F0BD8A0000208C0000204B
:1014C000891400004402002000B583B009236A4655
:1014D000137001335370013393700133D3700133B0
:1014E000137101335371034B98476B46185603B081
:1014F00000BDC0465114000010B5024B1B6800200F
:10150000984710BD8C00002010B5024B5B6801208D
:10151000984710BD8C00002010B5024B9B6802203C
:10152000984710BD8C00002010B5024BDB680320EB
:10153000984710BD8C00002010B5024B1B69042099
:10154000984710BD8C00002010B5024B5B69052048
:10155000984710BD8C0000200C4B1B68002B06D157
:10156000EFF31083002B07D00022094B1A70074AB3
:10157000136801331360704772B6BFF35F8F0022A8
:10158000044B1A700132024B1A70F0E7A4000020DD
:10159000A800002000000020084B1A68013A1A60D9
:1015A0001B68002B09D1064B1B78002B05D00122AC
:1015B000044B1A70BFF35F8F62B67047A40000201F
:1015C000A800002000000020F0B583B001AC012588
:1015D00065700027A770257021003E20064EB04799
:1015E0008022D205054B9A612770657021000F207B
:1015F000B04703B0F0BDC046011600008044004172
:1016000000B583B001AB80221A700A785A704A780C
:101610009A708A78DA701900014B984703B000BDC0
:10162000651B000010B5082803D880001C4B1B5810
:101630009F46002032E01B4B18692FE01A4B1B6AB3
:101640009B059B0F1948D84028E0164B586925E0A8
:10165000144B1B6800209B0720D513491022CB6830
:101660001A42FCD00F4B1A6824231340042B01D0DC
:101670000F4813E000200F4B98470A4B9B681B0450
:101680001B0C58430AE05023074AD35C00205B0739
:1016900004D5044BD86801E08020000210BDC0468C
:1016A000AC480000AC0000200008004000127A00A6
:1016B000006CDC02891A000070B50C490B6A0478D2
:1016C000857840780122104080014026B3430343CF
:1016D0002A40D20180208343134303222240120276
:1016E0000348034013430B6270BDC046000800402E
:1016F000FFFCFFFF082803D88000254B1B589F469E
:10170000172044E0234A136A02210B43136200208E
:101710003DE0204A936902210B439361002036E0AB
:101720001C4A138A02210B43138200202FE0194A1E
:10173000938A02210B439382002028E016490B680C
:10174000022213430B60134B9A8419000E32CB68AC
:101750001A42FCD0104A91680E4BD96252689A62C4
:1017600000229A8419001032CB681A42FCD00A4B2E
:101770001B689BB2074A9384002008E00549442275
:101780008B5C022003438B54002000E00020704754
:10179000D048000000080040AC00002030B585B003
:1017A000C222D2001A4B9A601A4A53681E218B43F8
:1017B000536001236A4613700024174DE0B2694656
:1017C000A8470134252CF9D103A800244470012531
:1017D00085700470114B98470620114B9847114BA8
:1017E0009847114B1C725C729C72DC7201956B46BF
:1017F0005C7006236A4613701472547269460020A6
:101800000A4B984700200A4B984705B030BDC046A8
:1018100000080040004000416D1A0000B9160000A9
:10182000F5160000351800000004004059180000AB
:1018300011190000064A936908210B4393610122A4
:10184000044B1A7019000B781342FCD17047C04644
:1018500000040040000C004070B5060004000D7844
:101860002D0205434B78002B02D08023DB021D4361
:101870004B7A002B02D080231B031D4348680128AC
:1018800010D9431E184234D1022830D90223002235
:1018900001325B009842FBD81202324314008023CD
:1018A0005B031D430B7A002B02D080239B031D4357
:1018B000134A53785BB2002BFBDB124B9847124B59
:1018C0001E700F4A53785BB2002BFBDB0C4B9C6005
:1018D0001A0053785BB2002BFBDB094A5368802166
:1018E00049020B401D435560084B984770BD0022CC
:1018F000D2E70402344380239B021D43D2E7C04653
:10190000000C004059150000080C0040991500001B
:1019100010B504000B4A53785BB2002BFBDB0A4B7B
:1019200098470A4B1C70074A53785BB2002BFBDBCD
:10193000044A516880235B020B435360044B984771
:1019400010BDC046000C004059150000040C0040BA
:101950009915000070B504001A4A53785BB2002B49
:10196000FBDB194B9847194B1C70164A53785BB236
:10197000002BFBDB134E7068C004C00E144B98475D
:101980000500124B1C707668F602F60F114B1C70A6
:101990000C4A53785BB2002BFBDB0A4B9C68240299
:1019A000240C0D4B9847002E07D1012C07D921009C
:1019B00028000A4B9847050001E00134E540280063
:1019C00070BDC046000C004059150000040C0040DA
:1019D00025160000080C004099150000451D000068
:1019E00010B50400064B9847064B1C70064A5388F6
:1019F0008021C9010B435380044B984710BDC0465A
:101A000059150000020C0040000C00409915000020
:101A100010B504000F4B98470F4B1C700F4A5388AA
:101A20001B05180F53880E490B40538053880D49EE
:101A30000B40538011008022D2014B881342FCD10D
:101A400006494A8803020648024013434B80064B6E
:101A5000984710BD59150000020C0040000C0040D2
:101A6000FFF0FFFFFFBFFFFF9915000010B50C78D6
:101A700024020443024B9847A4B2024B5C8010BD81
:101A8000111A0000000C004010B50400064B9847E6
:101A9000064B1C70064B5C882405240F054B9847A9
:101AA0002000054B984710BD59150000020C00405E
:101AB000000C0040991500005519000030B5D3788E
:101AC000002B35D11378802B29D01B06802464028B
:101AD000234354780225AC4306D19478002C20D1BE
:101AE0008024A402234341605478013C012C1CD97A
:101AF0000D042D0CA024E4052C431C4384620D0C22
:101B0000D02424062C431C438462D478002C22D198
:101B10005B031CD59378012B1ED0416117E0002395
:101B2000D7E7C024E4022343DDE70D4C2340DFE781
:101B300041600C04240CA023DB05234383620C0CBE
:101B4000D0231B0623438362D378002B03D1537821
:101B5000013B012B02D930BD8161F8E78160FAE7D2
:101B6000FFFFFBFF10B50A00C1090023002904D1C3
:101B70004309DB0105498C4663441F2420400121B1
:101B800081401800024B984710BDC04600440041F8
:101B9000BD1A00007047000010B5054B9847054B73
:101BA0009847054B9847054B9847054B984710BDFC
:101BB0009D170000C9150000951B0000951B000033
:101BC000951B0000FEE70000F8B52A4A2A4B9A420E
:101BD00011D01A00294B9A420DD2294A03339B1A7D
:101BE0009B0801339B000022234822498C588450D3
:101BF00004329A42FAD1234A234B9A420AD2D3435F
:101C000021495B1803218B4304339B18002102C236
:101C10009342FCD11D4AFF211D4B8B439360FD393C
:101C200090235B001B4AD1501B4AD3780325AB435A
:101C300002242343D370D3780C27BB4308263343B5
:101C4000D370164B987B3022904320221043987318
:101C5000997BB943314399739A7BAA4322439A7380
:101C60000F4A536880210B4353600E4B98470E4B2D
:101C70009847FEE7404A000000000020680000206E
:101C800004000020680000206002002000ED00E059
:101C90000000000000700041005000410048004179
:101CA0000040004179370000E91C00000300064AAB
:101CB0001268002A04D0044A1068C31813607047E1
:101CC0000249014A1160F6E7C400002060220020AA
:101CD00001204042704780239B014B6000207047E9
:101CE000012070470020704770B584B00F4B9847B3
:101CF0000F4B98470F4B98470F236B4400221A70E5
:101D0000019300240C4D0D4E02E00134772C0BD0D2
:101D10006B461C70012200216846A8470028F4D1B8
:101D200021000748B047F0E7FEE7C046991B0000D6
:101D3000B10A0000A909000021090000D137000004
:101D4000F4480000002243088B4274D303098B42FD
:101D50005FD3030A8B4244D3030B8B4228D3030C7B
:101D60008B420DD3FF22090212BA030C8B4202D31D
:101D70001212090265D0030B8B4219D300E0090A45
:101D8000C30B8B4201D3CB03C01A5241830B8B424E
:101D900001D38B03C01A5241430B8B4201D34B0337
:101DA000C01A5241030B8B4201D30B03C01A52419C
:101DB000C30A8B4201D3CB02C01A5241830A8B4221
:101DC00001D38B02C01A5241430A8B4201D34B020A
:101DD000C01A5241030A8B4201D30B02C01A52416E
:101DE000CDD2C3098B4201D3CB01C01A5241830922
:101DF0008B4201D38B01C01A524143098B4201D35C
:101E00004B01C01A524103098B4201D30B01C01A86
:101E10005241C3088B4201D3CB00C01A5241830800
:101E20008B4201D38B00C01A524143088B4201D32D
:101E30004B00C01A5241411A00D20146524110468D
:101E40007047FFE701B5002000F006F802BDC0466C
:101E50000029F7D076E770477047C046F0B5CE4608
:101E6000474615042D0C2E0080B50704140C3F0CBA
:101E70009946030C7E435D43674363437F19340CEB
:101E8000E4199C46A54203D980235B029846C444CA
:101E90004B46514343433604360C250C2404654419
:101EA000A4195918491920000CBC90469946F0BD58
:101EB000F8B54546DE4657464E460C03E0B54E00A3
:101EC000C90F88460D00610A440F0C43C70019036F
:101ED0005800DB0F9B464B0A510F0B43760D400D0C
:101EE0001900D200D84500D1AEE0351A002D00DC33
:101EF000F6E000280FD1134300D1DBE06B1E002B6E
:101F000000D037E1BA1A9742BF41641A7F42E41BFE
:101F10000126170024E0C64B9E424DD080231B04AF
:101F20001943382D00DD07E11F2D00DD38E12020A9
:101F3000431B9A460B00504683409946130048467F
:101F4000EB401843030050468240501E8241E94056
:101F50001A43BA1A611A9742A441170064420C1B33
:101F6000230262D56402650A002D00D1DFE028005B
:101F700001F0E4FB0300083B1F2B00DDD2E0202230
:101F80003C00D21A9D40D4409F4025439E4200DD34
:101F9000C4E09E1B731C1F2B00DDF1E020223800E3
:101FA0002900D21AD840914097402C000143781E56
:101FB0008741DC4000260F437B0709D00F233B40BD
:101FC000042B05D03B1DBB42BF417F42E4191F00DB
:101FD00023022CD5964B01369E4200D19AE045460D
:101FE000944BFF081C406007760564020743240BEE
:101FF000760D00212403230B0C0D8F4A24051C436E
:102000001440330523435B00ED075B082B43380086
:1020100019003CBC90469946A246AB46F8BD6446C2
:10202000044300D111E2040067467B07C6D1454650
:102030006007FF080743E4087D4B9E4230D024032D
:102040007605240B760DD4E7331A9A46002B78DDFB
:10205000002831D076488642AED08020000401436B
:102060005346382B00DCE9E00A43511E8A41002127
:10207000D219BA42BF4109197C4217000C19230238
:10208000D3D56B4B01369E4200D13AE10120694B1A
:102090001C407B0807401F43E007074364088BE7A9
:1020A00023003B4300D1CBE18022120314432403DD
:1020B000240B9EE72E007FE70800104300D1B4E018
:1020C000581E002800D0DEE0BA18BA429B416418BE
:1020D0005B42E418170001262302A6D50226D5E7A5
:1020E000002D6ED1701C4005400D012800DCF9E088
:1020F000B81A844687428041E51A40422D1A2802C8
:1021000000D489E0D71BBA4292411C1B5242A51A47
:10211000D84629E74546002400276AE7454CF61AC9
:102120002C4049E73D002838854000272EE738003D
:1021300001F004FB20301DE70A43511E8A410021B3
:1021400007E7002B00D0F3E0701C43055B0D012B6B
:1021500000DCADE0364B984200D1D1E0BA18BA426B
:10216000BF4164187F42E419E70752081743640827
:10217000060021E72E48854200D193E01D00D0E6FD
:1021800029001F3EF140202B00D18DE04022D31AC0
:102190009D402F437D1EAF4100240F43002644E79E
:1021A0002B000800203BD8400300202D00D17DE00B
:1021B0004020451BA9400A43511E8A4100211A4371
:1021C000C7E6002E50D01A4EB04257D080266B4240
:1021D0009946360434434B46382B00DDD6E01F2B9E
:1021E00000DD35E12026F51A2600AE40B2463E005D
:1021F000DE40AC46350056462E436546AF407D1E58
:10220000AF41DC403743D71BBA4292410C1B5242CC
:10221000A41A0600D846A3E6644667462C4300D0BD
:10222000A2E600250026002706E71E00C4E6C046F9
:10223000FF070000FFFF7FFFFFFF0F801F2B63DC06
:102240002020C31A080098409C468346534610003D
:10225000D84003005846184363469A40531E9A419B
:1022600053460243D94003E726003E4306D0EB43E2
:102270009946002BC7D0944EB042ACD10C00170049
:102280000600D84698E6904B9A450BD08246E7E682
:10229000002800D09EE01800104300D1E9E01C00A7
:1022A0001700D846884E87E6002572E7002182E7AE
:1022B00023003B43002E00D0ABE0002B00D1E7E031
:1022C0000B00134300D177E6BA18BA42BF41641835
:1022D0007F42E419230200D4F2E07C4B17001C403B
:1022E000060069E620003843002ED1D100285BD1DA
:1022F0001C00144300D1A8E01C001700D8465BE680
:1023000006000024002797E650460B002038C34003
:1023100099465346202B00D195E0402350461B1A86
:1023200099400A43511E8A414B4600211A439FE6B9
:10233000002E30D126003E4367D0DB439A46002B67
:102340001CD0614EB04260D05346382B00DD96E081
:102350001F2B00DD9FE02026F31A26009E409C469E
:10236000B34653463E00DE4033005E461E4363469E
:102370009F407B1E9F415346DC403743BF18974226
:10238000924164185242A418060078E627437C1E46
:10239000A741002437E74C4EB04236D080265B423E
:1023A00036049A463443CFE71800104300D103E6C1
:1023B000B81A84466745AD41E01A6D42401B0502DC
:1023C00000D42CE6D71BBA4292411C1B5242A41ADD
:1023D000D846F1E51800104300D163E7F808670715
:1023E00007438020E4080003044208D0DD080542CA
:1023F00005D1D208590711430F002C00D8467B0F96
:10240000E4001C43FF00304ED6E50C001700060028
:10241000D2E5002B38D00B00134300D142E7F80877
:10242000670707438020E40800030442E7D0CB0895
:102430000342E4D1D208490711430F001C00DEE734
:1024400000270024D5E500216BE700250027F3E5F0
:102450004E462500203EF5404B462E00202B2DD029
:102460004025ED1AAC4027437C1EA741002437438A
:10247000C9E6802400252403134E0027DCE527430A
:102480007C1EA741002479E70C0017000E4E93E54F
:102490000C00170090E556462300203EF340994675
:1024A0005346202B0ED0402356469B1B9C4027436F
:1024B0007C1EA7414B4600241F435FE70024D2E760
:1024C0001700B2E50024F2E7FF070000FFFF7FFFDF
:1024D000F0B557464546DE464E46E0B54C000E0385
:1024E00087B0834692461D008046360B640DCF0FA1
:1024F000002C4FD06F4B9C4235D08023420F1B04E1
:10250000F600134333439946C30098466A4B0026AE
:102510009C460023644403932B031B0B9B466B00D8
:10252000ED0F50465B0D01955ED0624A934253D049
:102530005A46D1008022400F120402430A439346B8
:102540005246D1005C4A94460022634438006840F9
:1025500084460290E41A16430F2E00D9B4E0574B7C
:10256000B6009B599F460300334399466CD1002324
:102570009846023308260393CEE7CB464146039A9A
:102580000197022A65D1019B4A4C9C4600230022F8
:1025900098466BE00300334399464ED0002E00D19D
:1025A000BCE1300001F0CAF803000B3B1C2B00DD3E
:1025B000ACE11D22D31A5A460100DA4008398E4098
:1025C0001300334399465B468B40984600233C4CAE
:1025D0000026241A03939FE751465A46114329D1F6
:1025E000002293460232B1E7594601431ED05B46B2
:1025F000002B00D19EE1584601F0A0F803000B3BF0
:102600001C2B00DD8FE102005946083A91408B46B1
:102610001D21CB1A5146D9400B0059460B43514658
:102620009B469140264B00221B1A8FE70023012274
:102630009B468BE75146032288E7002398460133E7
:1026400004260024039367E70323B14603930C2673
:1026500062E7032A00D15CE2019B012A00D0E4E199
:1026600013409C46002300240022984600211203B8
:10267000130B0A0D12051A432305124C4046224043
:10268000134362465B00D2075B081343190007B08F
:102690003CBC90469946A246AB46F0BD0023802242
:1026A0009C4612039846034CE0E70023014C0022AD
:1026B0009846DBE7FF07000001FCFFFF0849000028
:1026C0000DFCFFFFFFFF0F80D94500D939E100D194
:1026D00034E1002346464D469A46013C5B460A0ECD
:1026E0001B021A430B02170C039313041B0C390033
:1026F000280090460193FFF725FB0200019B8346CB
:102700005A43280039009146FFF7A2FB350C090413
:102710000D43A9450DD95B464544013BA84500D969
:102720003AE1A94500D837E102235B429C46454483
:10273000E3444B46EB1A390018000493FFF702FB01
:10274000019B05004343390004989946FFF780FB3D
:10275000330409041B0C0B43994509D943446A1EF1
:10276000984500D91AE1994500D817E1023D434444
:102770004A469B1A5A4612042A4303999346100C60
:102780000A0C914609045A46090C4E460D001204E3
:10279000120C4543059151437243704352190E0C7C
:1027A000B218954203D980256D02AC466044150CE1
:1027B00009041204090C28185218834200D2CEE0F2
:1027C00000D1C8E01D1A53469E1AB24592415242AA
:1027D000AB1A9A46984500D117E139001800FFF767
:1027E000B1FA019B05004343390050460493FFF7BB
:1027F0002FFB04980B04310C1943884209D941443A
:102800006B1E884500D907E1884200D804E1023DEB
:102810004144049BCB1A180039000493FFF792FA45
:10282000019B82464343390004980193FFF710FB54
:1028300001980B043104090C194388420DD9534601
:102840004144013B884500D9E8E0884200D8E5E0F2
:1028500002235B429C464144E244019B2D04CE1A74
:1028600051462943059D4F462A000B04080C1B0CBA
:102870005A4345437B4378435B19170CFB189D4231
:1028800003D980256D02AC4660441D0C12041B0464
:10289000120C28189B18864200D293E000D18EE0DB
:1028A00001231943A04BE318002B00DC99E04A07F1
:1028B00000D09EE05A46D20106D55A469B4B1A409C
:1028C00080239346DB00E318994A934268DD012395
:1028D000029A984C1A400023944698460022C5E676
:1028E00080224B46120313420AD05B46134206D1A4
:1028F0001A431203120BAC4688468E4CB6E64B4682
:102900001A431203120BBC468A4CAFE603005A4628
:10291000283B9A4000239146984657E6584600F0D7
:102920000DFF203040E603005246283B9A4000212C
:10293000934677E600F002FF20305FE6884500D23C
:10294000C7E64B46DE075D0843465B081E43434629
:10295000DB079A46C2E60025924500D333E7039E83
:102960005946B446E244B245AD416D424544EB1888
:102970000139984507D2984200D97FE000D1BCE0E8
:102980001D1A8B461FE79845FAD1039D5545F2D98C
:1029900043468B461D1A16E79B46CAE61500E7E636
:1029A0005A46C90852070A435B0590465C0D5A46D1
:1029B0000123029952021940120B8C4656E6002B55
:1029C00000D16FE746444A1EB04529D9110086421E
:1029D00000D065E7039A934200D061E762E70121E6
:1029E00049420120C21A382A21DD029B03409C463D
:1029F00038E60F220A40042A00D15BE70A00111DC5
:102A0000914292415242934454E7474BE318002BC2
:102A1000E5DD01225242F2E71D00FAE69A461CE784
:102A2000B04239D86ED011003AE702933AE71F2A34
:102A30003CDC20239B1A0C005846994098404B1EC2
:102A400099415B46D440D340204308431A004307D2
:102A500009D00F230340042B05D00100081D884234
:102A60009B415B42D21813023AD50123029A0124FA
:102A70001A400023944698460022F7E50221494275
:102A80008C46039DE344AC46E244AA45AD416D4209
:102A90004544ED182D1A96E68A1E03994D008D4285
:102AA000894149424144761803958FE71F204042EF
:102AB000C31A5846D8400300202A28D040205D463B
:102AC000821A954029434A1E914119430723002247
:102AD0000B4009D00F2300220B400800042BBDD16E
:102AE000010053075202120BC908194301238846FB
:102AF0000299002419408C46B8E55245BED88B4651
:102B0000002560E6039D9D42C6D3110062E70025C3
:102B1000D8E780225B4612031A43019B1203120B73
:102B20009C468846034CA1E5FF030000FFFFFFFE23
:102B3000FE070000FF070000F0B557464546DE4699
:102B40004E46E0B50C0398464E00230B87B00700B5
:102B500092469B46760DCD0F002E6BD06D4B9E425C
:102B600035D080245B46420F2404DB0014431C4311
:102B7000C3009946684BA3469C4600230027664441
:102B8000029343461C035A00DB0F5046240B520DA0
:102B9000984600D176E05F4B9A426DD08023410F7A
:102BA0001B040B435C49E4008C461C43C30000201B
:102BB00062444146B6186940721C0191944607432D
:102BC0000F2F00D9B0E0554ABF00D25997465B4657
:102BD0000343994600D087E000239B460233082731
:102BE0000293CEE742460192022867D0032800D123
:102BF0000EE2012800D062E1002300240022994661
:102C000001990140CDB2002112030B0D120B1B05DF
:102C10001343434A240513401C436400ED07640832
:102C20002C434846210007B03CBC90469946A2463A
:102C3000AB46F0BD034399464FD05B46002B00D115
:102C400089E1584600F07AFD03000B3B1C2B00DDA8
:102C50007AE11D22D31A3A0001005C46DA400839B5
:102C60008C4013008F4023439B46B94600232D4ED2
:102C70000027361A029384E7534623432AD10024BF
:102C8000022096E75346234320D0002C00D157E181
:102C9000200000F053FD03000B3B1C2B00DD49E13D
:102CA0001D21CB1A51460200D9405346083A9440A0
:102CB00093400C431B4A121A00207AE70125019B1E
:102CC000144C1D400023002299469CE7002400225A
:102CD00001206EE7534603206BE700239B46013338
:102CE0000427002602934CE7032381460C27029316
:102CF00047E780220023002512039946054C82E70E
:102D00005C464B4602986FE75C464B46019502983D
:102D10006AE7C046FF07000001FCFFFF48490000CA
:102D2000FFFF0F800DFCFFFF4A464946170C1A0CA7
:102D30001B041B0C08041900000C414315008846B5
:102D400019007D43794303958946290015004543C1
:102D50004D44029545462D0CAA46029D5544A94571
:102D600006D98A46802149028946CA4451460391C0
:102D7000290C0491414609042D04090C88462900B8
:102D8000250C24044144240C05912100414388462C
:102D9000210079438A466843414650448146080CE5
:102DA00048446F43824503D98021490289464F44F4
:102DB000010C894639004944029141460F040499A7
:102DC0003F0C88460004C01980444146049159468E
:102DD0000F0C0904090C884659438A4639005143AF
:102DE000894641464A435146090C8B467B43D218DB
:102DF0005A44934203D980235B029B46D9445146EF
:102E00000904090C8A46414661437C43130C1204B1
:102E10004B445244A1468A463C0041466C434D43D4
:102E200051464D440F0C7D19A94503D98021490213
:102E300088464444049F0399B84641448B468345E1
:102E4000804141428846514608042F04000C3F1837
:102E50005846029910188946904292414F44BA460A
:102E6000524299469346C244D144CB448F42BF411B
:102E7000C245894199459B41934592417F424942D0
:102E80002D0C52420F435B4213437F19FF185B46E0
:102E90003C19DB0D059A64021C43430213435D1E7B
:102EA000AB415A46C00D034352021343E20156D5CB
:102EB00001205A0803401343E207134364085A48A9
:102EC000604400284DDD5A0709D00F221A40042A19
:102ED00005D01A1D9A429B415B42E4181300E2019F
:102EE00004D58020514AC00014406044504A9042AA
:102EF00000DDE3E60125DB0862071A436402019B5B
:102F00009146220B4405640D1D407CE68022594603
:102F10001203114208D0144206D122431203120BAD
:102F200045469946434C6EE65B461A431203120B24
:102F3000404C68E603005446283B9C400023B9E619
:102F400000F0FCFB2030A6E60300283B9F40002356
:102F5000BB4699468AE600F0F1FB203074E6B446A1
:102F6000ADE701252A1A382A06DD019B00241D4001
:102F700000230022994646E61F2A21DC2025200056
:102F8000AD1A1E00AB40A840D6405D1EAB41304399
:102F90001843D440430709D00F230340042B05D026
:102FA0000300181D98429B415B42E418230221D57F
:102FB0000125019B01241D4000230022994622E6A1
:102FC0001F2521006D42281AC1400800202A1DD06B
:102FD0005F35AA1A944023435C1EA341072503438F
:102FE0001D400022002D09D00F2200241A40180095
:102FF000042AD6D1030065076402220BDB082B43A9
:1030000001259946019B00241D40FCE50024E2E7D0
:10301000802201251203224301991203120B0D4055
:103020009946044CEFE5C046FF030000FFFFFFFE9A
:10303000FE070000FF070000F0B54646D6464F46A3
:103040000C03C0B5CD0F4E00610A440F0C43C10004
:103050005800400D84468A460F001903500F490A54
:103060000143C648760DA846DB0FD200844500D147
:10307000D8E001204340AB4200D1A6E06046351ABB
:10308000002D00DC05E1002810D10B00134300D116
:10309000D7E06B1E002B00D04BE153469F1ABA4578
:1030A0008041641A4042241A01261EE0B34B9E421E
:1030B00048D080231B041943382D00DD19E11F2D52
:1030C00000DD4CE120230F005B1B10009A409F4065
:1030D000E840531E9A41E940074317435346DF1B1C
:1030E000611ABA45A44164420C1B230200D4C5E016
:1030F0006402650A002D00D1F6E0280000F01EFBF6
:103100000300083B1F2B00DDE9E020223C00D21A1F
:103110009D40D4409F4025439E4200DDDBE09E1B46
:10312000731C1F2B00DD0AE120223800D21A29006F
:1031300097402C009140D8407A1E9741DC400026F1
:1031400001430F437B0709D00F233B40042B05D0DD
:103150003B1DBB42BF417F42E4191F00230225D51E
:10316000864B01369E4200D1AFE0854B01251C40C5
:1031700043466207FF08640276051743240B760D69
:103180001D4000212403230B0C0D7E4A24051C4303
:103190001440330523435B00ED075B082B433800E5
:1031A00019001CBC90469946A246F0BD0125434635
:1031B0006207FF081743E4081D40704B9E4236D05B
:1031C00024037605240B760DDBE76346F31A002B08
:1031D00000DC94E06046002835D068488642B1D0D3
:1031E00080273F043943382B00DCFDE00A431700F9
:1031F00000217A1E9741574457458041091944429E
:103200000C1923023AD55D4B01369E4200D14BE1A9
:1032100001225B4B1C407B0817401F43E20717430A
:1032200064088FE70800104300D024E721E723005B
:103230003B4300D1B9E18022120314432403240B41
:103240009FE72E007EE70800104300D1CAE0581E19
:103250008446002800D0E7E052445245804164187B
:103260004042241817000126230207D50226CFE783
:1032700064462C4300D1B3E12C0067467B0700D0A5
:1032800062E76307FF081F4301254346E4081D402A
:1032900093E7002D78D1751C6D056D0D012D00DCB7
:1032A000F2E05046801A8245BF41651A7F42ED1B0D
:1032B0008446280200D48CE05046171ABA42924144
:1032C0000C1B5542651B984614E701254346002414
:1032D0001D40002755E72A4CF61A2C4032E73D00E6
:1032E00028388540002717E7380000F027FA2030FB
:1032F00006E70A43170000217A1E9741EEE6002BED
:1033000000D0E5E0731C9C465B055B0D012B00DCE7
:103310009FE01A4B9C4500D1C5E052445245804184
:10332000641840422418E7075208174364086646A9
:1033300008E71248854200D185E01D00BCE629005F
:103340001F3EF140202B00D17FE04022D31A9D4048
:103350002F437D1EAF4100240F4300268EE72B0034
:103360000F00203BDF40202D71D040235D1BA94082
:103370000A43511E8A4100211743AFE6FF070000B0
:10338000FFFF7FFFFFFF0F80002E3ED0B34EB445FE
:1033900045D0802636046D423443382D00DDA8E048
:1033A0001F2D00DD1FE1202627005046761BB74069
:1033B000E84007435046B040461EB041EC40384319
:1033C000171ABA4292410C1B5242A41A66469846FA
:1033D0008BE6644667462C4300D08BE6002500262A
:1033E0000027EAE61E00ADE61F2B60DC2027F81A56
:1033F0000F00844687401000D84007436046824053
:10340000501E8241D9401743F5E626005046064338
:1034100005D0ED43002DD3D0904EB445BDD10C0066
:103420001700664698468DE68C4883420BD063466B
:10343000D9E6002D00D096E00800104300D1E2E06C
:103440000C0017009846854E7CE6002580E7002199
:103450008EE7230050460343002E00D0A8E0002B47
:1034600000D1DEE00B00134300D16BE6524452451D
:1034700080416418404224181700230200D4FDE65E
:10348000774B66461C405DE6250050460543002EFE
:10349000CFD1002D4FD10C00144300D1A0E00C007F
:1034A000170098464EE666460024002785E61F0072
:1034B0000800203FF8400700202B00D18EE040207C
:1034C000C31A99400A43511E8A410021174392E6CC
:1034D000002E14D126005046064362D0DB43002B59
:1034E0005CD187189742924164185242A4186646EC
:1034F00087E650462043441EA041002460E7574E13
:10350000B4454ED0802636045B423443382B00DD70
:103510007FE01F2B00DD8BE0202627005046F61AA7
:10352000B740D84007435046B040461EB04107431D
:10353000DC40BF18D6E70D00154300D102E6504627
:10354000801A8245BF41651A7F42ED1B84462802DE
:1035500000D48DE65046171ABA4292410C1B5242D3
:10356000A41A9846EEE50D00154300D16BE75046CE
:103570006707C00807438020E4080003044207D01F
:10358000CD08054204D12C009846D70849070F43BF
:103590007B0FE4001C43FF00304ED3E52F4EB445B3
:1035A000B4D10C0017006646CCE500270024E8E5FE
:1035B000002B39D00B00134300D144E7C008670744
:1035C00007438020E40800030442E1D0CB08034213
:1035D000DED1D70849070F431C00D9E7002171E766
:1035E00000250027E9E52E002700203EF740202D8A
:1035F0002FD04026751BAC4050462043441EA041AE
:1036000000243843DCE6802400252403134E0027E1
:10361000D3E5504620430700781E87410024BF1899
:1036200060E70C0017008DE50C0017000B4E89E5D4
:103630001E002700203EF740202B0CD04026F31A16
:103640009C4050462043441EA04107430024BF181D
:1036500048E70024D0E70024F3E7C046FF07000056
:10366000FFFF7FFF30B5134D0A034B00120B5B0DBC
:10367000C90F0024AB4210DD0F4CA3420FDC8024A5
:103680000E4D64032243ED1A1F2D0BDD0C48C31AA7
:10369000DA405442002900D11400200030BD094B0B
:1036A000CC18FAE7084CE840A44663449A40024329
:1036B000EFE7C046FE0300001D04000033040000D5
:1036C00013040000FFFFFF7FEDFBFFFF10B5041E9A
:1036D00028D000F033F8154B154A1B1AD21A1F2AAE
:1036E00015DD144AD21A9440002224035B05240BF2
:1036F0005B0D0021100024030A0D240B1205224348
:103700000D4C1B05224013435B00590810BD2100DE
:1037100091400A000B21081AC4405B052403240BC6
:103720005B0DE6E7002300240022E2E71E04000010
:103730003304000013040000FFFF0F801C2101234D
:103740001B04984201D3000C10391B0A984201D384
:10375000000A08391B09984201D30009043902A262
:10376000105C40187047C0460403020201010101C9
:10377000000000000000000070B500260C4D0D4C4C
:10378000641BA410A64209D1002601F049F90A4D94
:103790000A4C641BA410A64205D170BDB300EB58BF
:1037A00098470136EEE7B300EB5898470136F2E749
:1037B0002C4A00002C4A00002C4A0000304A00002D
:1037C00003008218934200D1704719700133F9E762
:1037D0000FB40B4B13B51C68002C05D0A369002B4C
:1037E00002D1200000F0F2FA05AB049AA168200093
:1037F000019300F0C7FC16BC08BC04B01847C046D3
:103800000400002070B505000E00002804D0836974
:10381000002B01D100F0DAFAAB69AC68002B02D1C1
:10382000280000F0D3FA244B9C420FD16C68A38986
:103830001B0702D52369002B20D12100280000F0AE
:1038400057F900281AD00120404270BD1B4B9C4202
:1038500001D1AC68EBE71A4B9C42E8D1EC68E6E793
:10386000013B0136A360002B04DAA269934216DB08
:103870000A2914D023685A1C226019703178A36871
:103880000029EDD1013BA360002B0FDA22000A31A1
:10389000280000F0D7F8431CD5D00A20D5E7220035
:1038A000280000F0CFF8431CE8D1CCE70A202368B9
:1038B0005A1C22601870C8E7AC490000CC490000CF
:1038C0008C49000010B5034B01001868FFF79AFF00
:1038D00010BDC046040000204A424A41802310B572
:1038E0005200DB0000F002F810BD0000F0B51D0032
:1038F0004F4B85B01E6804000F000092002E05D0CB
:10390000B369002B02D1300000F060FA494B9C42B1
:1039100050D17468009B022B05D0012B00D984E0A4
:10392000002D00DA81E02100300000F0E1F9616B48
:10393000002908D023004433994202D0300000F01F
:1039400051FB002363630023A3616360A3891B060B
:1039500003D52169300000F045FBA389364A1340A6
:10396000A381009B022B5AD003AB02AA2100300096
:1039700000F0C2FAA3891843A081002D24D1029D32
:10398000280000F025FB0195071E42D1029B019300
:10399000AB4239D1012040420223A2891343A381C3
:1039A0000023A36023004733236023610123636165
:1039B00005B0F0BD214B9C4201D1B468AAE7204B71
:1039C0009C42A7D1F468A5E7002FD9D0B369002B9A
:1039D00002D1300000F0FAF9009B012B03D1A3893A
:1039E000009A1A43A2810820A38927602761656194
:1039F000184018D0012018400023984211D06D4281
:103A0000A360A5611800D3E7019800F0E1FA071E52
:103A1000C0D08023A289019D1343A381D6E7002053
:103A2000BAE7A560C4E7A060C2E701204042BFE753
:103A300004000020AC4900005CF3FFFFCC4900000B
:103A40008C490000F8B505000E001400002804D0D1
:103A50008369002B01D100F0B9F9224B9C422DD192
:103A60006C68A369A360A3891B0731D52369002B68
:103A70002ED023682269F7B2981A6369F6B2984289
:103A800005DB2100280000F033F9002826D1A368C7
:103A90000130013BA36023685A1C22601F706369D8
:103AA000984204D0A389DB071AD50A2E18D1210029
:103AB000280000F01DF9002812D00FE00A4B9C42AC
:103AC00001D1AC68CDE7094B9C42CAD1EC68C8E78C
:103AD0002100280000F00CF80028CAD00126764208
:103AE0003000F8BDAC490000CC4900008C49000012
:103AF000364B70B51D6806000C00002D05D0AB6973
:103B0000002B02D1280000F061F9314B9C420FD10B
:103B10006C680C23E25E93B219072DD4D90611D438
:103B200009230120336037331343A381404270BD22
:103B3000284B9C4201D1AC68EBE7274B9C42E8D173
:103B4000EC68E6E75B0713D5616B002908D023001A
:103B50004433994202D0300000F044FA00236363FA
:103B60002422A3899343A3810023636023692360F4
:103B70000823A2891343A3812369002B0BD1A02121
:103B80008022A389890092000B40934203D0210038
:103B9000300000F0D9F90123A289134011D000238D
:103BA000A36063695B42A361002023698342BED1A5
:103BB0000C23E25E1306BAD540231343A3810138D8
:103BC000B5E7920700D46369A360EDE70400002025
:103BD000AC490000CC4900008C490000F7B58A8947
:103BE00005000C00130760D44B68002B04DC0B6C41
:103BF000002B01DC0020FEBDE76A002FFAD0002375
:103C00002E682B6080235B011A4034D0606DA3893D
:103C10005B0706D56368C01A636B002B01D0236C69
:103C2000C01A0200216A00232800E76AB847A18968
:103C3000431C06D12B681D2B31D82C4ADA40D30700
:103C40002DD50023636023692360CB0405D5431C75
:103C500002D12B68002B00D16065616B2E600029BA
:103C6000C8D023004433994202D0280000F0BAF9AA
:103C700000206063BFE70123216A2800B847431C86
:103C8000C5D12B68002BC2D01D2B01D0162B01D122
:103C90002E60AFE74023A2891343A381ABE7402303
:103CA0000B430120A3814042A5E70F69002FA1D05B
:103CB0000B680F60DB1B01930023920700D14B6957
:103CC000A360019B002B00DC94E7019B3A00216A72
:103CD0002800A66AB047002803DC4023A2891343CA
:103CE000DFE7019B3F181B1A0193EAE70100402020
:103CF0000B6970B505000C00002B01D1002070BDD0
:103D0000002804D08369002B01D100F05FF80B4B31
:103D10009C4209D16C680C22A35E002BEED02100DE
:103D20002800FFF75BFFEAE7054B9C4201D1AC6836
:103D3000F1E7044B9C42EED1EC68ECE7AC490000A3
:103D4000CC4900008C49000010B5024900F0B2F8DF
:103D500010BDC046F13C0000002310B50400036014
:103D60004360836081814366C281036143618361F3
:103D7000190008225C30FFF723FD054B24626362C3
:103D8000044BA362044BE362044B236310BDC046A3
:103D9000F146000019470000514700007D47000030
:103DA00070B568254A1E55430E002900743100F095
:103DB00063F9041E08D000212A00016046600C301F
:103DC000A0606832FFF7FCFC200070BD836913B56A
:103DD0000400002B28D18364C3640365134B144A89
:103DE0001B6882620193984201D101238361200004
:103DF00000F020F86060200000F01CF8A0602000B7
:103E000000F018F80022E06004216068FFF7A4FFCA
:103E100001220921A068FFF79FFF02221221E0681A
:103E2000FFF79AFF0123A36113BDC0468849000034
:103E3000493D0000F8B51E4B07001E68B369002B12
:103E400002D13000FFF7C2FF4836B4687368013B07
:103E500004D53368002B07D03668F6E70C22A55E40
:103E6000002D0DD06834F2E704213800FFF798FFE9
:103E700030600028F0D10C2304003B602000F8BD26
:103E8000012320005B42E3810233A3816566256044
:103E9000A560656025616561A561082229005C3027
:103EA000FFF78EFC6563A563A564E564E6E7C0469D
:103EB00088490000F7B50400070000260191483446
:103EC000002C01D13000FEBD6368A5680093009B03
:103ED000013B009301D52468F2E7AB89012B08D997
:103EE0000E22AB5E013304D029003800019B9847B5
:103EF00006436835EBE7000070B50E001D000E2389
:103F0000C95E90B01400002907DA00232B60B38942
:103F10001B0611D48023DB000FE001AA00F05AFC3D
:103F20000028F2DBF022029B12021340054A9B1884
:103F30005A4253412B60EDE740230020236010B02C
:103F400070BDC04600E0FFFFF7B502268B89050073
:103F50000C00334206D02300473323602361012342
:103F60006361F7BD01AB6A46FFF7C6FF0099070022
:103F7000280000F081F8002808D10C22A35E9A05E1
:103F8000EFD4032293431E43A681E4E70F4BAB62B9
:103F90008023A28920601343A381009B2061636179
:103FA000019B002B0DD00E23E15E280000F024FCC5
:103FB000002806D00322A38993431A000123134348
:103FC000A381A0893843A081CBE7C046493D0000CA
:103FD00010B5034B0100186800F04EF810BDC04644
:103FE0000400002070B50500002910D00C1F2368C4
:103FF000002B00DAE418280000F02FFC1D4A13689B
:10400000002B05D163601460280000F027FC70BD10
:10401000A34209D9216860188342F3D118685B680C
:1040200041182160EEE713005A68002A01D0A2422D
:10403000F9D919685818A0420BD1206809185818E6
:1040400019608242E0D110685268411819605A60C4
:10405000DAE7A04202D90C232B60D5E7216860186B
:10406000824203D1106852684118216062605C602E
:10407000CAE7C046C8000020032370B5CD1C9D438D
:10408000083506000C2D1ED20C25A9421DD8300083
:1040900000F0E3FB254A14682100002919D1244CC3
:1040A0002368002B03D1300000F010FB20602900B2
:1040B000300000F00BFB431C2CD10C23300033608C
:1040C00000F0CCFB03E0002DDFDA0C23336000208E
:1040D00070BD0B685B1B1AD40B2B03D90B60CC187B
:1040E000256003E08C420ED163681360300000F05D
:1040F000B5FB200007220B30231D9043C31AE7D0E5
:104100005A42E250E4E74B6863600C00EEE70C00B3
:104110004968C2E70323C41C9C43A042E0D0211A93
:10412000300000F0D3FA431CDAD1C6E7C800002003
:10413000CC000020936810B5013B9360002B05DA9A
:104140009469A34208DBCBB20A2B05D01368581C34
:1041500010601970C8B210BDFFF774FCFBE7F8B52A
:1041600006000F001400D518AC4201D1002007E072
:1041700021783A003000FFF7DDFF0134431CF3D112
:10418000F8BD0000F0B59FB006000F0014000593C5
:10419000002804D08369002B01D1FFF717FE7F4B65
:1041A0009F425CD17768BB891B0762D53B69002BB6
:1041B0005FD0002306AD6B6120336B761033AB7696
:1041C0000294029C2378002B5DD1029BE31A049396
:1041D0000DD0049B029A39003000FFF7C0FF431C4A
:1041E00000D1CCE06A69049B944663446B612378F8
:1041F000002B00D1C3E00122002352426A6002A9D1
:104200005432521801342B60EB60AB601370AB6515
:1042100021780522624800F015FB631C9C460028AB
:1042200035D12968CB0604D5532302AA20309B1828
:1042300018700B0704D553232B2002AA9B18187063
:1042400023782A2B2CD000200A21099B2278303A8F
:10425000092A00D86BE000282AD0099328E0514BA6
:104260009F4201D1B7689EE74F4B9F429BD1F768B1
:1042700099E739003000FFF73BFC002899D0012076
:1042800040421FB0F0BD252B9FD001349AE7444B2C
:104290002968C01A012383400B432B606446B7E7AB
:1042A000059B181D1B680590002B3ADB099364469B
:1042B00023782E2B0BD16378621C2A2B3FD1059BD0
:1042C00002341A1D1B680592002B35DB07932178F9
:1042D0000322364800F0B6FA002807D0334B2A688C
:1042E000C01A4023834013432B6001342178631CA0
:1042F00006222F480293297600F0A4FA002844D021
:104300002C4B002B2FD12968059B0722C90528D5E6
:104310009B189343083305936B69039A9B186B6151
:104320004FE75B42EB6002230B432B60BFE74B433D
:1043300001349B18012089E701235B42C6E7002373
:1043400014000A201A006B6021783039092903D93A
:10435000002BBCD00792BAE7424301345218012324
:10436000F2E70733D5E705AB00933A00124B29007B
:10437000300000E000BF0390039B0133CCD1BB8928
:104380005B0600D57BE70B987BE705AB00933A0013
:10439000094B2900300000F07FF8ECE7AC49000041
:1043A000EC490000CC4900008C490000F2490000B3
:1043B000F6490000000000005F410000F7B515005D
:1043C00001938A680B6900900C00934200DA130095
:1043D00022002B6043321278002A01D001332B6077
:1043E00023689B0602D52B6802332B6006272368BF
:1043F0001F4027D0230043331B785A1E9341226865
:10440000920630D42200019943320098089EB047AA
:10441000431C25D0062320682A68E1680340002554
:10442000042B03D18D1AEB43DB171D40A3682269CF
:10443000934201DD9B1AED180027BD4220D10020D8
:1044400010E00137E3682A689B1A9F42D2DA220003
:104450000123193201990098089EB047431CF0D1FE
:1044600001204042FEBD3020E11843310870210098
:104470005A1C45310978A218433202331170C1E742
:10448000220001231A3201990098089EB047431C6C
:10449000E6D00137D1E70000F0B58BB006920A00F4
:1044A00043320793059004920A7E0C00109B6E2AFB
:1044B00000D18FE017D8632A2CD008D8002A00D169
:1044C00099E0582A54D026004236327029E0642AF6
:1044D00001D0692AF7D121681A68080623D5111D71
:1044E0001960156825E0732A00D188E008D86F2A82
:1044F00029D0702AE7D1202209680A43226003E00C
:10450000752A20D0782ADED1220078214532117018
:104510006C4A30E00E001A684236111D19601368AB
:104520003370012379E04906D9D5111D19600023A4
:10453000D55E002D03DA2D23049A6D421370624B71
:104540000A2703932FE020681968050603D5081D84
:1045500018600D6805E04006F9D50D68081D186063
:10456000ADB2594B082703936F2A18D00A2716E0DB
:1045700045310A70544A03921A682168101D186068
:104580001568080622D5CB0702D5202319432160E0
:104590001027002D03D1202322689A432260230094
:1045A000002243331A706368A360002B5CDB042293
:1045B000216891432160002D58D1049E002B64D0C6
:1045C0002600039B42361B7833705EE04806DAD53E
:1045D000ADB2D8E709681A68080605D5111D19603B
:1045E000136862691A6006E04906F7D5111D196063
:1045F0001368A28A1A800023049E236154E01A687B
:10460000111D1960166800216268300000F01AF967
:10461000002801D0801B6060636823610023049A36
:10462000137041E02369320006990598079DA84759
:10463000431C43D0236800259B070FD4099BE068E7
:1046400098423DDA18003BE0220001231932069916
:104650000598079EB047431C30D00135E368099A9E
:104660009B1A9D42F0DBE9E7002DA9D0049E2800AB
:104670003900FDF7EDFB039B013E5B5C28003370C6
:104680003900FDF75FFB051EF1D1082F09D1236822
:10469000DB0706D563682269934202DC3023013EC2
:1046A0003370049B9B1B2361079B09AA0093210085
:1046B000069B0598FFF782FE431CB3D101204042C0
:1046C0000BB0F0BD0E4A0000FD490000002370B59C
:1046D000064C050008002360FDF7E8FA431C03D1EF
:1046E0002368002B00D02B6070BDC0465C02002008
:1046F00070B50C000E25495F00F0B2F8002803DB0E
:10470000636D1B18636570BDA389024A1340A381C2
:10471000F9E7C046FFEFFFFFF8B51F008B890500E2
:104720000C001600DB0505D50E23C95E002202230E
:1047300000F074F8A389054A28001340A3813200D1
:104740000E23E15E3B0000F01FF8F8BDFFEFFFFF16
:1047500070B50C000E25495F00F060F8A389421C7B
:1047600003D1054A1340A38170BD80225201134337
:10477000A3816065F8E7C046FFEFFFFF10B50E2389
:10478000C95E00F015F810BD70B5050008001100F5
:104790000022064C22601A00FCF79AF8431C03D151
:1047A0002368002B00D02B6070BDC0465C02002047
:1047B000002370B5064C050008002360FDF788FA59
:1047C000431C03D12368002B00D02B6070BDC04672
:1047D0005C020020002370B5064C050008001100A3
:1047E0002360FDF778FA431C03D12368002B00D027
:1047F0002B6070BD5C020020002370B5064C0500E4
:1048000008002360FDF76CFA431C03D12368002BDA
:1048100000D02B6070BDC0465C02002070B5050062
:10482000080011000022064C22601A00FDF75AFA17
:10483000431C03D12368002B00D02B6070BDC04601
:104840005C020020C9B28218904201D1002070475A
:1048500003788B42FBD00130F6E7704770470000C9
:1048600070B50500080011000022064C22601A00F5
:10487000FCF70CF8431C03D12368002B00D02B60FD
:1048800070BDC0465C02002048656C6C6F20776F7D
:10489000726C640000080042000C004200100042EC
:1048A0000014004200180042001C004236160000AE
:1048B000321600003216000098160000981600000C
:1048C0004A1600003C160000501600008616000034
:1048D0002017000000170000001700008C170000D0
:1048E000121700002E170000041700003C170000EC
:1048F0007C17000049324320616464726573732041
:104900003078253032780A00C8260000AA26000038
:104910006426000082250000642600009C2600001A
:104920006426000082250000AA260000AA260000B6
:104930009C260000822500007A2500007A250000D0
:104940007A250000E0280000282D0000E82B000058
:10495000E82B0000E42B0000002D0000002D0000DB
:10496000F22C0000E42B0000002D0000F22C0000CF
:10497000002D0000E42B0000082D0000082D000091
:10498000082D00000C2F000008000020000000008F
:104990000000000000000000000000000000000017
:1049A0000000000000000000000000000000000007
:1049B00000000000000000000000000000000000F7
:1049C00000000000000000000000000000000000E7
:1049D00000000000000000000000000000000000D7
:1049E000000000000000000000000000232D302B1C
:1049F0002000686C4C0065666745464700303132E0
:104A00003334353637383941424344454600303136
:104A10003233343536373839616263646566000095
:104A2000F8B5C046F8BC08BC9E467047DD000000E3
:104A3000F8B5C046F8BC08BC9E467047B5000000FB
:104A4000010000000800002000000000AC49000048
:104A5000CC4900008C49000000000000000000006C
:104A60000000000000000000000000000000000046
:104A70000000000000000000000000000000000036
:104A80000000000000000000000000000000000026
:104A90000000000000000000000000000000000016
:084AA00000000000000000000E
:0400000300001BC915
:00000001FF
